:020000040000FA
:040000000000B9291A
:080008008B138C106D088316A8
:1000100092008312EC0BB7290230EC006E08031932
:100020003328DE01EE191B286E192128EE18272827
:100030006E182D287C2905191F28DE151628EE11AB
:100040001428051D25285E1516286E1116288519F9
:100050002B28DE147C29EE101828851D31285E140B
:100060007C296E107C29671844280508033965022D
:10007000031D3E28E90BC928E714C928671403307B
:10008000E8000F30E900C928E80BC92800308A00D1
:1000900005080339E600E50D650D0C3966070F39D3
:1000A000820761289E2866286128662861286128C1
:1000B0009E289E28612861286628612866289E2837
:1000C0006128671005080339E500C92805080339C8
:1000D000E500E71C6D2801306E280830EB00E701D1
:1000E000D807031C75280130D90720085802DA0008
:1000F000031C7C2800307D28013021075902DB00D9
:10010000031C86285A08D8005B08D9006B08D20760
:10011000031C8C280130D30720085202DA00031C8C
:10012000932800309428013021075302DB00031C80
:10013000C9285A08D2005B08D300C928050803392A
:10014000E500E71CA5280130A6280830EB00E701F0
:10015000D8020318B8280130D9020318B82820089B
:10016000D807031CB5280130B62800302107D9076D
:100170006B08D2020318C9280130D3020318C9281A
:100180002008D207031CC6280130C72800302107E9
:10019000D307DE0152085002DA00031CD5285308A9
:1001A0005102DB00031CDB28E52801305307510214
:1001B000DB000318E528DE14DB09DA090130DA0771
:1001C000031CEF280130DB07EF285E14DA08031D5B
:1001D000EF28DB08031DEF28DE105E1023295A08E4
:1001E0002202031CF8285B082302031CFE280029B6
:1001F00001305B072302031CFE2800290330DE06C2
:10020000DE1C1329D208031D0D29D308031D0D2957
:100210002008D2002108D30023290130D20203187C
:100220002329D302232920085202031D1E29210855
:100230005302031D1E29D201D30123290130D20705
:10024000031C2329D30756085402DA00031C2E2965
:1002500057085502DB00031C34293E29013057079B
:100260005502DB0003183E29DE15DB09DA090130EF
:10027000DA07031C48290130DB0748295E15DA0834
:10028000031D4829DB08031D4829DE115E117C2966
:100290005A082602031C51295B082702031C572910
:1002A000592901305B072702031C572959290C30B3
:1002B000DE06DE1D6C29D608031D6629D708031D3E
:1002C00066292408D6002508D7007C290130D602EB
:1002D00003187C29D7027C2924085602031D77299C
:1002E00021085702031D7729D601D7017C29013047
:1002F000D607031C7C29D7075E080319B729DE1926
:10030000DD035E19DD0ADE18DC035E18DC0A01304D
:100310008A005C0807398E21DF009729820708349C
:100320000A3402340634043405340134093401300B
:100330008A005D0807399E21DF04A72982078034DF
:10034000A0342034603440345034103490340830B9
:10035000E00006138612DF1FAF290616B229061227
:10036000000000008616DF0DE00BAA2906178B1788
:1003700009000F30EE004130C0000030BD00E63013
:10038000ED000230EC000030C100C200C300C40028
:10039000C500C600C700C800D200D300D600D700F1
:1003A000D000D100D400D500D800D900DC00DD0099
:1003B000BE01E3012030B8008312B901380884007F
:1003C0003908840783169B001C141A0883128000C6
:1003D000B90A0F303902031DDE295A30B200B300CA
:1003E000B4003930B500B6003230B000B101293068
:1003F000B800B901BA01BB01BD0107309F008316E7
:100400000F308600FF30850083128316E93092009A
:1004100083120730920083164D30990020309800E7
:100420008312903098008B170B1783168C1483124D
:100430008B178C1A1E2AE31B282B192A8B131A08D8
:10044000BC008C123B18732ABA1B4D2A300884005A
:100450003108840700083C02031D382AB10A053020
:100460003102031D392AB101B901FF30BA00182A3F
:10047000B101380884003908840700083C02031DD4
:100480004B2AB90A05303902031D182AB101B901F6
:10049000FF30BA00182AB901182A3C08BA00FF3008
:1004A000BB0002308A003A080F396222CD004D08A5
:1004B0000319812ABD01EA01CD1F182ACD1328088E
:1004C000EA00182A820700340434843406340134E4
:1004D000003400340034003405340834013400346E
:1004E000003400340034EA080319782AEA03182A91
:1004F000400884003D0884073C088000BD0ACD0BFD
:10050000182ABD01BB0102308A003A080F39820760
:10051000B929982A982AB929B929E22AB929B929E1
:10052000E82AFA2ACA2AF02AB929B929B929B929FF
:1005300041082002031CA12A42082102031CAC2A04
:10054000A72A013042072102031CAC2AA72A41082E
:10055000D0004208D100B12A2008D0002108D100E3
:10056000B12A43082402031CBA2A44082502031CAA
:10057000C52AC02A013044072502031CC52AC02A07
:100580004308D4004408D500182A2408D4002508BC
:10059000D500182A4108A0004208A1004308A20083
:1005A0004408A3004508A4004608A5004708A60083
:1005B0004808A7000030E2002030E1000830E000E9
:1005C000BA010B2B580899008030E300BA01182AB1
:1005D0000830E2001130E4008130E300BA01182A4B
:1005E0004108A8000830E2002830E1000130E000B6
:1005F000BA010B2B4108A9004208AA004308AB002E
:100600004408AC004508AD000930E2002930E100A3
:100610000530E000BA0161088400000883169A00E2
:100620008312620883169B009C111C1555309D0097
:10063000AA309D009C141C1183128C1F1D2B8C133F
:10064000E20AE10AE00B0B2BB901BA01BB01182A3F
:100650008B130C1E182A631C392B620883169B000F
:100660001C141A0883129900E20AE40B182AE30109
:0A067000182A59089900E301182A1E
:02400E00613F10
:10420000A0000500D0000200A0000500D0000200C0
:10421000000045004E0047003900390020005300DF
:104220005400450050002000560031002E003000A0
:04423000300030002A
:00000001FF
